S01100004D49432D5765656B312E7372656350
S113000045C0000060C000005EC000005CC000008D
S11300105AC0000058C0000056C0000054C0000080
S113002052C0000050C000004EC000004CC0000090
S11300304AC0000048C0000046C0000044C00000A0
S113004043C0000040C000003EC000003CC00000AF
S11300503AC0000038C0000036C0000034C00000C0
S113006032C0000030C000002EC000002CC00000D0
S11300702AC0000028C0000026C0000024C00000E0
S113008022C0000020C000001EC0000011241FBEBA
S1130090CFEFD0E1DEBFCDBF11E0A0E0B1E0E4E1FD
S11300A0F2E000E00BBF02C007900D92A230B1074E
S11300B0D9F721E0A2E0B1E001C01D92A830B20757
S11300C0E1F799D0A5C09CCF1F920F920FB60F9263
S11300D011242F938F939F93989B1AC080910401AE
S11300E090910501892BA1F4809100019091010167
S11300F0880F991F909301018093000181E090E0A3
S11301009093070180930601909305018093040165
S1130110999B1DC08091020190910301892BB9F430
S1130120809100019091010199230CF40196959519
S11301308795909301018093000181E090E0909372
S1130140070180930601909303018093020183B316
S1130150811108C01092050110920401109203014C
S11301601092020180910001909101018431910566
S11301703CF484E190E0909301018093000109C074
S1130180813A9F4034F080EA9FE09093010180938C
S113019000019F918F912F910F900FBE0F901F9090
S11301A01895989B05C083E081BB81E082BB0895CC
S11301B0999B05C083E081BB82E082BB08959A9B32
S11301C005C086E081BB82E082BB08959B9B05C08D
S11301D086E081BB84E082BB08959C9B05C085E0DA
S11301E081BB84E082BB08959D9B04C085E081BBF4
S11301F081E082BB089514BA8FEF81BB83B783601B
S113020083BF87B7816087BF12BE7894CADFFECFF1
S1070210F894FFCF8C
S1050214E803F9
S9030000FC
